:100000000C94D3020C9417030C9417030C9417034D
:100010000C9417030C9417030C9417030C941703F8
:100020000C9417030C9417030C94CF0D0C94A10E91
:100030000C9417030C9417030C9417030C941703D8
:100040000C9417030C94AB220C9417030C94170315
:100050000C9417030C943E1C0C9417030C94170378
:100060000C9417030C9417030C9417030C941703A8
:100070000C9417030C9417030C9417030C94170398
:100080000C9417030C9417030C9417030C94170388
:100090000C9417030C9417030C9417030C94170378
:1000A0000C9417030C9417030C9417030E0F300FC6
:1000B0001E10300F1E10750F980F1E10ED0F001040
:1000C000CF12CF12FE12FE1234135413851485146E
:1000D0005F1385140F140F147614851485147F1480
:1000E0001C141C141C141C141C141C141C141C1490
:1000F0001C141C141C141C141C141C141C141C1480
:100100002E143B14421449145314750A01E2012CB5
:10011000022C02E2746401160216010402040109B1
:1001200002090104020401150215010C020C012848
:10013000022800750A01E2012C022C02E27464011B
:10014000170217010802080115021501100210011B
:100150000C020C0111021101040204010F020F0133
:1001600028022800750A01E2012C022C02E27464C4
:100170000105020501050205010802080107020741
:10018000010C020C011702170128022800750A0150
:10019000E30116021602E301E3012B022B02E30145
:1001A000E30115021502E300750A01E301160216C8
:1001B00002E301E3012B022B02E3000000F0A12E79
:1001C000004C002A00E100E00000001E00140004C2
:1001D000001D00E200E2001F001A0016001B00E3F1
:1001E000002A00200008000700060050002C002113
:1001F000001500090019004F004B00220017000AEB
:1002000000050000003500015401520000E3000029
:10021000003400015401520000E3000000290023D3
:10022000001C000B00110000002A00240018000D23
:1002300000100052004E0025000C000E0036005148
:10024000002800260012000F0037002F002B002787
:10025000001300334238713000E0002D00310034CB
:1002600078E5002C00000001000100010001000100
:100270000000003A002F0036020100010001003B9F
:1002800000300037020100010001003C002F02266F
:10029000020100010001003D0030022702010001BF
:1002A0000001003E003402340001000000010001A2
:1002B0000001000000010000000100010001000039
:1002C000000100000001003F0038002D0024020062
:1002D0000001004000240021001E0027004A0041C8
:1002E00000250022001F00370001004200260023E5
:1002F00000200050000100430025022E022E004F76
:10030000004D004400450001000100010000000113
:10031000000100010001000100000069000100016E
:10032000000100010001006A000100043001000129
:1003300000010001004B004E00010001000100011E
:100340000001300100010001004A000100033001FA
:100350000002300000010001000100000001000067
:100360000001001408010000000100000001001A53
:100370000830082F082C0200000100350A520C50EA
:10038000002C00A9000100350852005100AC00AA61
:100390000019080100510C4F00AB00A8000608012D
:1003A0000001000100010001001B08A5000100AED2
:1003B0000001000100000016034500720067006F95
:1003C0000044006F007800200045005A000000162D
:1003D000034500720067006F0044006F0078002042
:1003E0000045005A0000000403090409026D0004DE
:1003F0000100A0FA09040000010301010009211114
:10040000010001223F000705810308000A090401D9
:10041000000103010200092111010001224D000722
:1004200005820308000A0904020001030000000914
:1004300021110100012236000705830308000A0983
:100440000403000103000000092111010001223909
:1004500000070584031000011201100100000008CC
:10046000EDFE071301000102000105010906A101CB
:10047000050719E029E71500250195087501810296
:100480000508190129059505750191029501750366
:100490009101050719002977150025019578750147
:1004A0008102C005010980A101850216010026B75D
:1004B000001A01002AB700751095018100C0050CD3
:1004C0000901A1018503160100269C021A01002AD8
:1004D0009C02751095018100C005010902A1010966
:1004E00001A10005091901290515002501950575CA
:1004F000018102950175038101050109300931155A
:1005000081257F95027508810609381581257F951B
:100510000175088106050C0A38021581257F9501B1
:1005200075088106C0C005010906A101050719E08B
:1005300029E71500250195087501810295017508C7
:10054000810105081901290595057501910295019B
:10055000750391010507190029FF150025FF950670
:1005600075088100C00000000000000000000000CD
:10057000010204060A0F17202C3A4A5D71879DB3C9
:10058000C7DAE9F5FCFFFCF5E9DAC7B39D87715DD1
:100590004A3A2C20170F0A0604020100000000004E
:1005A00000000000000011241FBECFEFDAE0DEBF24
:1005B000CDBF04B603FE24C08091FB019091FC01E5
:1005C000A091FD01B091FE018730904BA740B04B48
:1005D000B9F41092FB011092FC011092FD011092EF
:1005E000FE0114BE84B7877F84BF88E10FB6F894FC
:1005F00080936000109260000FBEE0E0FFE3099579
:1006000011E0A0E0B1E0E4EEF8E402C005900D9244
:10061000A433B107D9F711E0A4E3B1E001C01D9202
:10062000AB3FB107E1F70E94130B0C9470240C94BC
:100630000000FC016230B9F028F4662341F061301B
:1006400061F023C06330A9F06430C9F01EC082811C
:100650008823D9F088EA91E0089582818823A9F05F
:100660008DE891E008958281882379F084E691E015
:1006700008958281882349F083E391E0089582817F
:10068000882319F08AE091E0089580E090E00895D1
:1006900008956091BD017091BE018091BF0190915C
:1006A000C0010E94701B56985E9825982D98269838
:1006B0002E9827982F98813019F0823021F00895D4
:1006C000259A2D9A0895269A2E9A08950C944903F6
:1006D00056985E9825982D9826982E9827982F98AA
:1006E0008FEF90E0909389008093880090938B0027
:1006F00080938A0090938D0080938C00259A2D9A88
:100700002FEF80E792E0215080409040E1F700C059
:100710000000269A2E9A2FEF80E792E02150804029
:100720009040E1F700C00000279A2F9A2FEF80E752
:1007300092E0215080409040E1F700C000002598F1
:100740002D982FEF80E792E0215080409040E1F714
:1007500000C0000026982E982FEF80E792E02150ED
:1007600080409040E1F700C0000027982F985698ED
:100770005E9825982D9826982E9827982F9808955A
:1007800089EA8093800089E08093810024982C98E6
:100790003F988AB18F748AB96E98479A8BB1806BF3
:1007A0008BB9769A0E9468030C94480380E2809388
:1007B00000018091340181110EC00E94250481E066
:1007C000809334012FEF83ED90E3215080409040DF
:1007D000E1F700C0000080E40E942B048093000138
:1007E00081112EC00E94550480930001811128C000
:1007F0000E94550480930001811122C08FE30E9462
:1008000055048093000181111BC00E944D0480E4B7
:100810000E942B0480930001811112C08CE00E9481
:1008200055048093000181110BC00E9455048093F0
:100830000001811105C08FE30E94550480930001DF
:100840000E944D048091000108951092B9008AE041
:100850008093B800089594EA9093BC009091BC00F6
:1008600097FFFCCF9091B900987F983021F090319C
:1008700011F081E008958093BB0084E88093BC0070
:100880008091BC0087FFFCCF8091B900887F8831C0
:1008900011F0803471F780E0089584E98093BC0002
:1008A0008091BC0084FDFCCF08958093BB0084E858
:1008B0008093BC008091BC0087FFFCCF9091B90071
:1008C000987F81E0983209F480E0089584E880936D
:1008D000BC008091BC0087FFFCCF8091BB000895D5
:1008E00080910001811115C080E40E942B04809347
:1008F000000181110CC082E10E9455048093000127
:10090000811105C08FEF0E945504809300010E9461
:100910004D0484B1807F84B985B1807F85B98AB167
:10092000837F8AB98BB1837F8BB93E9846980895AF
:100930000E94D603809300010E94700480B38C70E3
:1009400080BB81B3836F81BBA6E3B1E0E4E4F1E057
:100950008EE08E0F11921D928E13FCCF0C94C0036B
:10096000BF92CF92DF92EF92FF920F931F93CF939C
:10097000DF9380910001882379F0809135018F5FAA
:1009800080933501811108C00E94D6038093000135
:10099000811102C00E94680306E311E0C0E0D0E0CC
:1009A000DD24D39482E0C82EEE24E394F12CC730EA
:1009B000D10500F580910001811164C080E40E949E
:1009C0002B0480930001811112C082E10E94550422
:1009D0008093000181110BC0C7010C2E01C0880F4C
:1009E0000A94EAF780950E945504809300010E94C2
:1009F0004D0448C0CA30A1F028F4C83059F0C930BD
:100A000061F005C0CC3089F070F0CD3089F0209ACB
:100A1000289810C0219A29980DC0229A2A980AC0B5
:100A2000239A2B9807C0529A01C0539A5B9802C030
:100A30003E9A469890EA9A95F1F79FB1799902C04B
:100A400082E001C080E091709D25982B7C9902C0C6
:100A500084E001C080E0892B7D9902C038E001C0AC
:100A600030E0832B7E9902C020E101C020E0822B80
:100A70009FB19095991F9927991F9295990F907EF4
:100A8000892B0FC080910001811149C080E40E9430
:100A90002B0480930001882379F1B12C0E944D042E
:100AA0008B2DF8019081981719F08083C092010175
:100AB0000E94700421960F5F1F4FCE30D10509F0C0
:100AC00076CF80910101882361F1815080930101EB
:100AD000882339F08FE99FE00197F1F700C000000B
:100AE00020C0A4E4B1E0E6E3F1E0CF01825F9191A0
:100AF0009D938E13FCCF15C083E10E945504809313
:100B000000018111CACF81E40E942B04809300016F
:100B10008111C3CF0E946604B82EB094BFCF80E08D
:100B2000C0CF0E94660381E0DF91CF911F910F91AA
:100B3000FF90EF90DF90CF90BF900895E82FF0E006
:100B4000EC5BFE4F8081089508950F931F93CF9320
:100B5000DF93C4E4D1E010E00C2F025F899190E0B4
:100B60000E94641B180F0C13F9CF812FDF91CF91D6
:100B70001F910F91089581E0089508950F931F9399
:100B8000CF93DF938C01FC01C081D181CE010E9403
:100B9000E919BE010E946106EC01F80182818823F7
:100BA00009F44AC080915D0181111FC0C431F0E594
:100BB000DF0709F051C00E94BD0581E080935D010F
:100BC0000E94081C90935C0180935B011092540179
:100BD000109256011092550110925801109257012F
:100BE00010925A011092590165C080915B01909159
:100BF0005C010E94141C883C910570F480915401A2
:100C0000E82FF0E0EE0FFF1FEB5AFE4FD183C083B9
:100C10008F5F809354014EC0C43880E5D80721F01F
:100C2000C538D04501F13AC0F8018281882341F0EE
:100C30001092520182E01EC0C438E0E5DE0759F58B
:100C400080915201811106C086E20E94731186E2F2
:100C50000E943B1282E01CC0C438F0E5DF0741F37C
:100C6000C538D045D9F4F8018281882331F010923B
:100C7000530180E20E948A121DC0809153018111AC
:100C800006C087E20E94731187E20E943B1280E255
:100C90000E9491120FC0C538D04529F381E080939E
:100CA000520180935301C801DF91CF911F910F91A1
:100CB0000C94BB0580E0DF91CF911F910F910895B7
:100CC000089596E0799FF001112494E5899FE00D45
:100CD000F11D1124E60FF11DEE0FFF1FE154FE4F31
:100CE000859194910895880F991FFC01E55CFF4F51
:100CF000859194910895880F991FFC01E554FE4F4A
:100D00008591949108950F931F93CF93DF93EC01F6
:100D10008115904350F5C11580E2D80708F0C3C093
:100D2000CB3BD10590F4C83AD10508F06AC0C53A6A
:100D3000D10508F05BC0C430D10508F0D0C12197BF
:100D400009F0CAC101E010E00AC2CF3FD10511F09D
:100D500008F0C5C1C03FD10508F0A2C0CE01805E39
:100D60009109089708F4BBC1B7C1C13090E5D90714
:100D700009F4A2C020F5C0318FE4D80770F4C11582
:100D800090E4D90708F094C0C11521E3D20708F018
:100D9000A3C1DD278E01106CE2C1C115D04509F059
:100DA0009BC10E94F0148FEF94E32CE0815090409F
:100DB0002040E1F700C000000E94631CD0C1C115B3
:100DC00097E5D90758F4C03121E5D20708F01CC1D6
:100DD000C43180E5D80708F475C07EC1CE019057B4
:100DE0008115904108F078C1DF7073C1C53AD10513
:100DF00009F477C1C63AD10509F076C102E810E4DA
:100E0000AEC1C83AD10509F472C1C93AD10509F495
:100E100071C1CA3AD10509F470C1CB3AD10509F4C0
:100E20006FC1CC3AD10509F46EC1CD3AD10509F4B0
:100E30006DC1C03BD10509F46CC1CE3AD10509F4AE
:100E40006BC1CF3AD10509F46AC1C13BD10509F4A0
:100E500069C1C23BD10509F468C1C33BD10509F49E
:100E600067C1C43BD10509F466C1C53BD10509F48E
:100E700065C1C63BD10509F464C1C73BD10509F47E
:100E800063C1C83BD10509F462C1C93BD10509F46E
:100E900061C1CA3BD10509F460C100E014E45FC13F
:100EA0008E0110655CC1CE019F700E947B0658C107
:100EB000DF708E01106A53C18091DA0181608093E6
:100EC000DA014DC10E94081E811102C00E94EE1D70
:100ED0000E94251E90E09093FB018093FA01C2309E
:100EE00080E5D80721F48091FA01816086C0C43082
:100EF00090E5D90721F48091FA0182607EC0C63066
:100F000020E5D20721F48091FA01846076C0C830D0
:100F100080E5D80719F48091FA0127C0CA3090E51E
:100F2000D90721F48091FA01806167C0CC3020E5B7
:100F3000D20721F48091FA0180625FC0CE3080E553
:100F4000D80721F48091FA01806457C0C03190E540
:100F5000D90721F48091FA0180684FC0C23120E5A1
:100F6000D20729F48091FA018460886046C0C330BA
:100F700080E5D80721F48091FA018E7F3EC0C5300C
:100F800090E5D90721F48091FA018D7F36C0C730F2
:100F900020E5D20721F48091FA018B7F2EC0C93061
:100FA00080E5D80719F48091FA0126C0CB3090E58E
:100FB000D90721F48091FA018F7E1FC0CD3020E542
:100FC000D20721F48091FA018F7D17C0CF3080E5E0
:100FD000D80721F48091FA018F7B0FC0C13190E5D1
:100FE000D90721F48091FA018F7707C0C331D0452A
:100FF00031F48091FA018B7F877F8093FA01809191
:10100000FA010E94291EABC08D2F99278F70992756
:1010100081309105D9F49E012370332702C0880FD7
:10102000991F2A95E2F79C688E0144E0000F111F7A
:101030004A95E1F700271370802B912B53E0CC0FDA
:10104000DD1F5A95E1F7C076DD272FC0823091056C
:1010500031F4DC2FCC278E01016F106A80C0833001
:10106000910569F4CE018370992701E010E002C078
:10107000000F111F8A95E2F7C8019C680FC08430E9
:101080009105B9F4CE018370992701E010E002C008
:10109000000F111F8A95E2F7C8019A6823E0CC0F70
:1010A000DD1F2A95E1F7C07ED7708C010C2B1D2B1C
:1010B00056C08530910531F4DC2FCC278E01046FAA
:1010C000106A4DC0069709F04AC0CF71DD27DC2FAA
:1010D000CC278E01106243C000E010E040C08E01BA
:1010E0003EC001E810E43BC003E810E438C002EE63
:1010F00014E435C009EE14E432C00AEE14E42FC043
:1011000005EB14E42CC006EB14E429C007EB14E44F
:1011100026C00CEC14E423C00DEC14E420C003E85A
:1011200015E41DC00AE815E41AC002E915E417C069
:1011300004E915E414C001E216E411C003E216E468
:101140000EC004E216E40BC005E216E408C006E295
:1011500016E405C007E216E402C00AE216E4C8017C
:10116000DF91CF911F910F91089596E0799FF00143
:10117000112494E5899FE00DF11D1124E60FF11D66
:10118000EE0FFF1FE154FE4F85919491803E910533
:10119000E0F4803C910558F58133910509F46FC066
:1011A00048F48932910509F463C08A32910509F443
:1011B0006DC072C089339105E9F082389105D1F094
:1011C0008533910509F44DC067C0833E910581F1D7
:1011D00038F4803E9105B9F0823E9105D9F05CC0AB
:1011E000863E910561F1873E9105A1F155C00E94AF
:1011F000730608952091FA0120FD02C021FF4CC022
:1012000080EE90E049C08091FA0180FFF9CF89E338
:1012100090E042C08091FA0182FF0EC08091FA01F5
:1012200084FF03C080E090E037C083EE90E034C0DC
:101230008091FA0182FFF2CF82EE90E02DC0809182
:10124000FA0183FF0BC08091FA0184FDEBCF87EE9A
:1012500090E022C08091FA0183FFF5CF86EE90E006
:101260001BC08091FA0185FF07C089E290E014C09D
:101270008091FA0185FFF9CF85E390E00DC0809160
:10128000FA0186FF07C08AE290E006C08091FA0169
:1012900086FFF9CF81E390E00E94830608950895C8
:1012A0000C944F0980916E010895CF93DF9300D085
:1012B0001F92CDB7DEB79C018091F101843019F502
:1012C00093E099833B832A839093E9008FEF909179
:1012D000E800815095FD06C095ED9A95F1F7000064
:1012E0008111F5CF8091E80085FF0DC040E050E00E
:1012F00063E070E0CE0101960E94BF0B8091E80090
:101300008E778093E8000F900F900F90DF91CF9130
:101310000895CF93DF9300D01F92CDB7DEB7209111
:10132000F101243021F522E029839B838A8383E025
:101330008093E9008FEF9091E800815095FD06C001
:1013400095ED9A95F1F700008111F5CF8091E800B5
:1013500085FF0DC040E050E063E070E0CE010196F3
:101360000E94BF0B8091E8008E778093E8000F9079
:101370000F900F90DF91CF9108952091F1012430CB
:10138000F1F422E02093E9002FEF3091E8002150A2
:1013900035FD06C035ED3A95F1F700002111F5CF86
:1013A0002091E80025FF0BC040E050E065E070E0D0
:1013B0000E94BF0B8091E8008E778093E80008952B
:1013C000CF93DF93EC019091F101943009F046C086
:1013D00080910C018823D9F080910D018823B9F008
:1013E0009093E9008FEF9091E800815095FD06C041
:1013F00095E19A95F1F700008111F5CF8091E80011
:1014000085FF2CC040E050E060E170E017C081E053
:101410008093E9008FEF9091E800815095FD06C020
:1014200095ED9A95F1F700008111F5CF8091E800D4
:1014300085FF14C040E050E068E070E0CE010E94FB
:10144000BF0B8091E8008E778093E80080E1FE0179
:10145000AEE5B1E001900D928A95E1F7DF91CF9171
:1014600008958091F001811109C00E94540D0E94DD
:10147000B10D8091E20084608093E20008951092A3
:10148000F001089508950C9498220E94F91B0E947F
:101490009E220E9457100C94500942E061EC81E0BA
:1014A0000E94CE0C42E061EC82E00E94CE0C42E051
:1014B00061EC83E00E94CE0C42E161EC84E00C948C
:1014C000CE0C8091F301833009F455C030F48130A3
:1014D00071F0823009F48EC008958A3009F47AC020
:1014E0008B3009F460C0893009F09CC020C0809125
:1014F000F201813A09F096C08091E800877F8093DD
:10150000E8008091F6019091F701892B21F460E1C8
:101510008EE591E003C060E080E090E070E00E9422
:101520000A0C8091E8008B778093E8000895809101
:10153000F201813209F076C08091F6019091F701B5
:10154000009719F0039709F06DC08091E800877F3C
:101550008093E8008091E80082FD05C08091F10150
:101560008111F8CF5FC08091F10080936E0180916E
:10157000E8008B7753C08091F201813A09F052C0A4
:101580008091F6019091F701892B09F04BC0809171
:10159000E800877F8093E8008091E80080FFFCCF1F
:1015A00080910C0136C08091F2018132D9F5809191
:1015B000F6019091F701892BA9F58091E800877FCA
:1015C0008093E8000E94030D8091F40180930C0148
:1015D0000C94F0148091F201813221F58091E800A1
:1015E000877F8093E8000E94030D8091F50180932E
:1015F0006F0108958091F201813AA1F48091E80091
:10160000877F8093E8008091E80080FFFCCF809185
:101610006F018093F1008091E8008E778093E8005D
:101620000C94030D089584B7877F84BF88E10FB6BB
:10163000F89480936000109260000FBE90E080E804
:101640000FB6F89480936100909361000FBE0E94E2
:10165000A6100E94540D0E94B10D8091E20084609A
:101660008093E20078940E9437100E94A81082E0D4
:1016700091E00E9452100E9486228091F1018530F3
:1016800069F40E94C01B8091EF018823B1F30E948E
:10169000EB1B882391F30E94A90BEFCF0E94AE10A1
:1016A000ECCF292F332723303105C9F064F42130E2
:1016B000310581F02230310509F043C08DE690E01C
:1016C0002BEE33E042C021323105F1F022323105F8
:1016D00041F137C082E190E028E534E036C0992737
:1016E0008130910541F08230910541F0892B49F517
:1016F000E7EEF3E005C0EFECF3E002C0E7EBF3E068
:10170000849190E09F0121C06430D8F4E62FF0E08E
:10171000EE0FFF1FEE5DFE4F2081318189E090E0EA
:1017200014C0643070F470E0FB01EE0FFF1FE65E42
:10173000FE4F20813181FB01EA5EFE4F808190E007
:1017400004C080E090E020E030E0FA0131832083A3
:10175000089580E189BD82E189BD09B400FEFDCF15
:101760008091D8008F7D8093D8008091E0008260C6
:101770008093E0008091E00081FDFCCF0895CF923E
:10178000DF92EF92FF920F931F93CF93DF93EC01C1
:101790008B016A010E94220D811133C0C114D10452
:1017A00039F0F60180819181081B190BC80FD91FF0
:1017B000E12CF12C0115110519F18091E80085FD4E
:1017C00016C08091E8008E778093E800C114D104A0
:1017D00049F0F60180819181E80EF91EF182E082E4
:1017E00085E00FC00E94220D882321F30AC0899151
:1017F0008093F10001501109FFEFEF1AFF0ADACFD1
:1018000080E0DF91CF911F910F91FF90EF90DF90DB
:10181000CF9008952091F8013091F90126173707EC
:1018200048F06115710539F42091E8002E77209376
:10183000E80001C0B90140E061157105A9F12091EE
:10184000F101222309F443C0253009F442C020915C
:10185000E80023FD40C02091E80022FD32C0209125
:10186000E80020FFE9CF4091F3002091F20030E042
:10187000342BFC01CF016115710559F02830310579
:1018800040F481918093F100615071092F5F3F4FC7
:10189000F1CF41E02830310509F040E02091E80027
:1018A0002E772093E800C8CF4111C9CF0AC080919C
:1018B000F101882361F0853061F08091E80083FDBB
:1018C0000AC08091E80082FFF2CF80E0089582E0B4
:1018D000089583E0089581E008952091F801309102
:1018E000F9012617370748F06115710539F4209181
:1018F000E8002E772093E80001C0B901FC0120E048
:101900006115710591F18091F101882309F440C0BE
:10191000853009F43FC08091E80083FD3DC080918F
:10192000E80082FD2FC08091E80080FFE9CF209180
:10193000F3008091F20090E0922B6115710559F04F
:101940008830910540F424912093F1003196615044
:1019500071090196F2CF21E0089709F020E080910B
:10196000E8008E778093E800CBCF2111CCCF0AC05E
:101970008091F101882361F0853061F08091E80069
:1019800083FD0AC08091E80082FFF2CF80E00895D5
:1019900082E0089583E0089581E00895982F9730BC
:1019A00058F59093E900981739F07091EC00209168
:1019B000ED005091F00003C0242F762F50E021FF5E
:1019C00019C03091EB003E7F3093EB003091ED0079
:1019D0003D7F3093ED003091EB0031603093EB00B0
:1019E0007093EC002093ED005093F0002091EE00F6
:1019F00027FF07C09F5FD3CF8F708093E90081E0FE
:101A0000089580E008958091F20187FF11C08091D0
:101A1000E80082FD05C08091F1018111F8CF11C06D
:101A20008091E8008B770BC08091F101882349F009
:101A30008091E80080FFF8CF8091E8008E77809356
:101A4000E80008952091E4003091E50095E640918A
:101A5000EC00842F817040FF22C08091E80080FD5F
:101A60001CC08091F101882391F0853091F0809124
:101A7000EB0085FD10C04091E4005091E500421755
:101A8000530729F39A01915011F784E0089582E0F9
:101A9000089583E0089581E0089580E008954091DD
:101AA000E80042FFDECF08950E94C20D0E94CA0DD9
:101AB000E0EEF0E0808181608083E8EDF0E08081FD
:101AC0008F77808319BCA7EDB0E08C918E7F8C93CB
:101AD00080818F7E80831092F00108950F931F9371
:101AE000CF93DF930E94C20D0E94CA0DC8EDD0E0D3
:101AF00088818F77888388818068888388818F7DBB
:101B0000888319BC1092F1011092ED011092EF013F
:101B10001092EE0100EE10E0F80180818B7F80834F
:101B200088818160888342E060E080E00E94CE0C82
:101B3000E1EEF0E080818E7F8083E2EEF0E0808154
:101B400081608083808188608083F80180818E7FBE
:101B50008083888180618883DF91CF911F910F916D
:101B60000895E8EDF0E080818F7E8083E7EDF0E07E
:101B700080818160808384E082BF81E08093F00176
:101B80000C946E0DE8EDF0E080818E7F80831092E2
:101B9000E20008951092DA001092E10008951F9279
:101BA0000F920FB60F9211242F933F934F935F9391
:101BB0006F937F938F939F93AF93BF93EF93FF9315
:101BC0008091E10082FF0BC08091E20082FF07C09C
:101BD0008091E1008B7F8093E1000E94361080911C
:101BE000DA0080FF1FC08091D80080FF1BC0809169
:101BF000DA008E7F8093DA008091D90080FF0DC0DB
:101C000080E189BD82E189BD09B400FEFDCF81E09C
:101C10008093F1010E94310A05C019BC1092F101B4
:101C20000E943F0A8091E10080FF19C08091E2008C
:101C300080FF15C08091E2008E7F8093E20080914A
:101C4000E20080618093E2008091D80080628093FE
:101C5000D80019BC85E08093F1010E94430A80916D
:101C6000E10084FF30C08091E20084FF2CC080E15D
:101C700089BD82E189BD09B400FEFDCF8091D80005
:101C80008F7D8093D8008091E1008F7E8093E1006A
:101C90008091E2008F7E8093E2008091E20081607B
:101CA0008093E2008091ED01882311F084E007C069
:101CB0008091E30087FD02C081E001C083E0809352
:101CC000F1010E94450A8091E10083FF29C08091C3
:101CD000E20083FF25C08091E100877F8093E100CF
:101CE00082E08093F1011092ED018091E1008E7FFE
:101CF0008093E1008091E2008E7F8093E2008091EA
:101D0000E20080618093E20042E060E080E00E94B7
:101D1000CE0C8091F00088608093F0000E94420A0F
:101D2000FF91EF91BF91AF919F918F917F916F91B3
:101D30005F914F913F912F910F900FBE0F901F9089
:101D400018951F920F920FB60F9211242F933F9365
:101D50004F935F936F937F938F939F93AF93BF93B3
:101D6000CF93DF93EF93FF93C091E900CF70809101
:101D7000EC00D82FD17080FDD0E81092E90080915E
:101D8000F000877F8093F00078940E94E50E109217
:101D9000E9008091F00088608093F000CD2BCF7037
:101DA000C093E900FF91EF91DF91CF91BF91AF9187
:101DB0009F918F917F916F915F914F913F912F9163
:101DC0000F900FBE0F901F9018951F93CF93DF9326
:101DD000CDB7DEB7AA970FB6F894DEBF0FBECDBF62
:101DE000E2EFF1E088E08E0F9091F10091938E1375
:101DF000FBCF0E94610A8091E80083FF1FC18091A0
:101E0000F2019091F301492F50E04A30510508F05A
:101E100015C1FA01EA5AFF4F0C942024803881F052
:101E2000823809F00BC18091F6018F708093E90030
:101E30008091EB0085FB882780F91092E90006C0AD
:101E40008091EE019091EF01911182609091E800F4
:101E5000977F9093E8008093F1001092F100C8C042
:101E6000282F2D7F09F0EAC0882319F0823061F015
:101E7000E5C08091F401813009F0E0C0933009F0B1
:101E800080E08093EF012BC08091F401811127C085
:101E90008091F6018F7009F4D1C08093E900209100
:101EA000EB0020FF1CC0933021F48091EB00806296
:101EB00014C09091EB0090619093EB0021E030E032
:101EC000A90102C0440F551F8A95E2F74093EA002A
:101ED0001092EA008091EB0088608093EB001092F2
:101EE000E9008091E800877F86C08111A7C010912A
:101EF000F4011F778091E3008078812B8093E300C9
:101F00008091E800877F8093E8000E94030D809114
:101F1000E80080FFFCCF8091E30080688093E300BD
:101F2000111102C082E001C083E08093F10186C0FC
:101F30008058823008F082C08091F4019091F501C0
:101F40008C3D53E0950779F583E08A838AE28983A3
:101F50004FB7F894DE01139620E03EE051E2E32F04
:101F6000F0E050935700E49120FF03C0E295EF703A
:101F70003F5FEF708E2F90E0EA3010F0C79601C0FF
:101F8000C0968D939D932F5F243149F74FBF809169
:101F9000E800877F8093E8006AE270E0CE01019656
:101FA0000E940A0C14C0AE014F5F5F4F6091F601B2
:101FB0000E94510BBC01892B09F440C09091E800AC
:101FC000977F9093E80089819A810E946D0C80919F
:101FD000E8008B778093E80031C0803879F58091F4
:101FE000E800877F8093E8008091ED018093F10005
:101FF0008091E8008E778093E8000E94030D1EC058
:1020000081111CC09091F4019230C0F48091E800DD
:10201000877F8093E8009093ED010E94030D8091EB
:10202000ED01811106C08091E30087FD02C081E0CF
:1020300001C084E08093F1010E944D0A8091E80084
:1020400083FF0AC08091E800877F8093E800809139
:10205000EB0080628093EB00AA960FB6F894DEBF87
:102060000FBECDBFDF91CF911F9108950895CF93FB
:102070008091F1018823A1F0C091E900CF70909187
:10208000EC00892F817090FD80E8C82B1092E90048
:102090008091E80083FD0E94E50ECF70C093E900B7
:1020A000CF91089590937501809374010895E09104
:1020B0007401F0917501309721F00190F081E02DCD
:1020C000099480E00895E0917401F09175013097D2
:1020D00021F00280F381E02D09940895E0917401CC
:1020E000F0917501309721F00480F581E02D09947D
:1020F000089520917201309173018217930771F056
:102100009093730180937201E0917401F0917501D5
:10211000309721F00680F781E02D099408952091F1
:102120007001309171018217930771F090937101E2
:1021300080937001E0917401F0917501309721F066
:102140000084F185E02D0994089508950C94A5105C
:102150000E94FF1B0E9498040C94C11C9F92AF9296
:10216000BF92CF92DF92EF92FF920F931F93CF9384
:10217000DF9300D000D000D0CDB7DEB70E94B0040E
:102180000DE010E0AA24A394B12C902E802F0E9481
:102190009E05980129583E4F6901F901F080F82603
:1021A000A1F40150110988F78FEF89838A831B827C
:1021B0000E94081C8160782F9D838C8349815A81FD
:1021C0006B818D810E9445112FC09091DA0191FFA2
:1021D00004C08E830E94A4058E8125E030E0A50115
:1021E000022E01C0440F0A94EAF7E42E4F21C1F0F9
:1021F00029839A828E2191E009F490E09B830E94CA
:10220000081C8160782F9D838C8349815A816B8162
:102210008D810E944511F6018081E826E08204C08C
:1022200021503109E0F6BDCF0E94A81F1091760120
:102230000E9457101817B9F00E945710809376012A
:1022400026960FB6F894DEBF0FBECDBFDF91CF91BB
:102250001F910F91FF90EF90DF90CF90BF90AF90C4
:102260009F900C94500926960FB6F894DEBF0FBECF
:10227000CDBFDF91CF911F910F91FF90EF90DF9035
:10228000CF90BF90AF909F900895CF93DF93CDB73D
:10229000DEB72B970FB6F894DEBF0FBECDBF4F83CE
:1022A000588769877A878B87DE01119686E0FD0162
:1022B00011928A95E9F785E0FE01379601900D921B
:1022C0008A95E1F749815A816B817C818D819E815C
:1022D0000E948E172B960FB6F894DEBF0FBECDBFAF
:1022E000DF91CF910895CF93882309F4C2C0C82FFE
:1022F000823859F40E94571081FDBBC089E30E94C7
:10230000681A0E94351B89E30CC0833879F40E9457
:10231000571080FDAEC083E50E94681A0E94351BED
:1023200083E50E94AA1ACF910C94351B843859F486
:102330000E94571082FD9DC087E40E94681A0E9487
:10234000351B87E4EECF8CEF8C0F813A48F48C2F4D
:102350000E94EB2181118DC08C2F0E94681AE3CF5F
:1023600080E28C0F883048F4C77081E001C0880F8C
:10237000CA95EAF70E94EE1AD6CF8BE58C0F833010
:1023800078F4C53A29F0C63A31F083E890E005C008
:1023900081E890E002C082E890E0CF910C9479103F
:1023A00088E58C0F833108F064C0C83A39F1C93A26
:1023B00041F1CA3A49F1CB3A51F1CC3A59F1CD3A0F
:1023C00061F1C03B69F1CE3A71F1CF3A79F1C13B8D
:1023D00081F1C23B89F1C33B91F1C43B99F1C53B0B
:1023E000A1F1C63BA9F1C73BB1F1C83BB9F1C93B6B
:1023F000C1F1CA3BC9F180E090E038C082EE90E0C4
:1024000035C089EE90E032C08AEE90E02FC085EBB7
:1024100090E02CC086EB90E029C087EB90E026C0CE
:102420008CEC90E023C08DEC90E020C083E891E03C
:102430001DC08AE891E01AC082E991E017C084E9E2
:1024400091E014C081E292E011C083E292E00EC0FC
:1024500084E292E00BC085E292E008C086E292E05E
:1024600005C087E292E002C08AE292E0CF910C942C
:102470008F10CF910895882309F44BC0823859F406
:102480000E94571081FF45C089E30E94681A0E948C
:10249000351B89E30CC0833871F40E94571080FF0C
:1024A00038C083E50E94681A0E94351B83E50E94AC
:1024B000AA1A0C94351B843859F40E94571082FFD5
:1024C00028C087E40E94681A0E94351B87E4EFCF7A
:1024D0009CEF980F913A58F390E2980F983050F48F
:1024E000877091E001C0990F8A95EAF7892F0E94C1
:1024F000F41ADFCF9BE5980F933020F480E090E052
:102500000C947910885A833120F480E090E00C9488
:102510008F100895882321F00E94EE1A0C94351B29
:102520000895882321F00E94F41A0C94351B089515
:102530007F928F929F92AF92BF92CF92DF92EF9253
:10254000FF920F931F93CF93DF931F92CDB7DEB708
:102550007C01C62E772EFC01058102950F70128139
:1025600011110E940B1B0E94611A882379F011231C
:1025700069F080E28C0D883048F082E00E944A1AAF
:102580000E94611A91E0D82ED92601C0D12CE72DE6
:10259000E295EF70F0E0E05AFF4F0C942024872D75
:1025A000807F072D0F70882311F00295007F112383
:1025B00089F0002309F490C180E28C0D883020F46A
:1025C000802F0E94EE1A03C0802F0E94FE1A0E94E4
:1025D000351B82C18C2D0E943B12002309F495C14A
:1025E00080E28C0D883020F4802F0E94F41A03C002
:1025F000802F0E94041B0E94351B87C1972D907F5E
:10260000872D8F70903211F08295807FCC2021F041
:10261000F1E0CF16B1F01EC0112349F0002309F4F8
:1026200014C1013009F011C10E941E1B6EC10023AC
:1026300019F0013009F469C189830E94211B898145
:102640000AC1112321F0023008F05FC1FEC0011160
:102650005CC101C1112321F0002309F4F6C03CC183
:10266000002309F4F8C03EC1872D869586958370B6
:1026700090E0009719F0019761F047C1112321F014
:102680008C2D972D937002C080E090E00E9479100D
:102690003CC1112321F08C2D972D937002C080E056
:1026A00090E00E948F1031C18C2D112319F00E94EF
:1026B000B01E02C00E94181F0E949D1F26C1872DB8
:1026C000837009F052C0111120C18C2D829586951E
:1026D0008770880F880F9C2D9F70892E912CA12CBC
:1026E000B12C082E04C0880C991CAA1CBB1C0A948F
:1026F000D2F7C4FE14C00FE010E020E030E0B901D2
:10270000A80104C0440F551F661F771F8A95D2F792
:10271000CB01BA01609570958095909503C060E0FB
:1027200070E0CB01272D26952695237030E02230CE
:10273000310569F02330310589F0682979298A2922
:102740009B292130310571F00E94D618DEC068291E
:1027500079298A299B290E94F218D7C00E94D6188D
:10276000C501B4010E94BA18D0C0112319F0872DF9
:10277000817001C08695882309F4C7C08C2D82958D
:1027800086958770880F880F9C2D9F70892E912CBD
:10279000A12CB12C082E04C0880C991CAA1CBB1CAF
:1027A0000A94D2F7C4FE14C00FE010E020E030E03D
:1027B000B901A80104C0440F551F661F771F8A95F1
:1027C000D2F7CB01BA01609570958095909503C0C2
:1027D00060E070E0CB01272D269526952370422FCF
:1027E00050E04230510569F04330510589F06829C5
:1027F00079298A299B294130510571F00E94B0192D
:1028000084C0682979298A299B290E94CC197DC016
:102810000E94B019C501B4010E94941976C08C2D94
:1028200090E0FC01E05EF109E531F10508F050C0EF
:10283000E059FF4F0C9420240C2D0F70872D8F71C1
:10284000112331F00E942D19802F0E948A125DC041
:102850000E944E19802F0E94911257C0112339F007
:10286000011153C0872D8F710E9473194EC0023021
:1028700008F04BC0F7CF112339F0872D8F710E94DC
:102880002D1943C01123C9F3872D8F710E944E1952
:102890003CC0112329F0872D8F710E94181935C073
:1028A0000E940E1932C0112351F0172D1F71812F74
:1028B0000E942D1963E0812F0E94411A26C081E0F9
:1028C0000E944A1A023008F182E00E944A1A1DC092
:1028D000112331F0002389F28C2D0E94731115C051
:1028E000002391F28C2D0E943B120FC0472D4F7098
:1028F0006C2DC7010E9419030E94321806C0472D93
:102900004F706C2DC7010E946006DD20F9F00E9417
:102910003D1A80FD1BC0F70112820E94371A0E94E7
:102920002D19C7010E94B5140E94371A0F90DF912C
:10293000CF911F910F91FF90EF90DF90CF90BF90BC
:10294000AF909F908F907F900C944E190F90DF91D5
:10295000CF911F910F91FF90EF90DF90CF90BF909C
:10296000AF909F908F907F9008950F931F93CF9378
:10297000DF93EC01888199812B813C81232BB9F075
:102980009F3F11F48F3F99F0CE010E94BE0588232E
:1029900071F0688179818A810E94331A8C010E94CA
:1029A000E8190E94AF18B801CE010E949812DF9179
:1029B000CF911F910F9108950E940B1B0E941B1B2A
:1029C0000E94E01A0E94351B0E944E200E949D1F0B
:1029D00080E090E00E94791080E090E00C948F10ED
:1029E0000E94FB1A0C94DC140E94281A292F2295AD
:1029F0002F7030E02C3031054CF42A3031056CF466
:102A00002250310922303105A8F407C02C3031059D
:102A100069F02F30310551F00DC0803F69F018F496
:102A2000803E40F409C0843F29F406C093FB882708
:102A300080F9089580E0089581E00895CF93DF93B1
:102A400000D000D01F92CDB7DEB70F900F900F903F
:102A50000F900F90DF91CF910895CF93DF9300D027
:102A600000D000D0CDB7DEB726960FB6F894DEBF03
:102A70000FBECDBFDF91CF9108951F93CF93DF930A
:102A8000C091850116E080918601C81799F0D0E0C9
:102A90001C9FF0011D9FF00D1124E957FE4F40814E
:102AA000518162817381848195810E942D152196C7
:102AB000C770E9CFDF91CF911F9108954091B70181
:102AC0005091B8016091B9017091BA018091BB0138
:102AD0009091BC010C942D158091BC0182958F7052
:102AE00009F054C08091B901882309F44FC0809146
:102AF0008501A09186016091B7017091B801409164
:102B0000BA015091BB01B6E08A1709F43FC090E0CA
:102B100041155105C1F17F3F11F46F3FA1F1B89FFD
:102B2000F001B99FF00D1124E957FE4F2181721376
:102B30002AC02081621327C02281211124C0238151
:102B400034812417350710F421503109241B350B2B
:102B5000283C3105C0F42091BC012F7020612093E6
:102B6000BC0126E0289FF001299FF00D1124E457B5
:102B7000FE4F80818F708061808387EB91E00E949F
:102B8000B5140C943D1501968770BECF0895CF9271
:102B9000DF92EF92FF920F931F93CF93DF93CDB706
:102BA000DEB762970FB6F894DEBF0FBECDBF8C01C3
:102BB00085E0F801DE011D9601900D928A95E1F7FE
:102BC000D8014C9111965C91119712966C911297C5
:102BD0001396CD90DC9014973091B7017091B801A5
:102BE0008091BA019091BB01009709F46BC17F3FBE
:102BF00019F43F3F09F466C1E090B901EE2009F4F1
:102C0000C0C02091BC01C816D90628F0F601E81B07
:102C1000F90BCF0104C0809590958C0D9D1DFF246C
:102C2000F394883C910578F0F12C207F09F0C6C020
:102C30007C2DD98AC88A89890E941E1587EB91E06C
:102C40000E94B514B1C0822F807F09F046C0751371
:102C500014C0341312C0611110C02F702061209372
:102C6000BC010E945E1587EB91E00E94B514809133
:102C7000BC01D80115968C932EC0CD2819F15F3F69
:102C800011F44F3FF9F0F62E61111CC080918501BF
:102C90002091860136E0821709F45AC090E0389FEF
:102CA000F001399FF00D1124E957FE4F7181571340
:102CB00006C07081471303C07281711103C0019671
:102CC0008770E9CFF62E662309F418C18091BC0104
:102CD00081608093BC01F12C11C1751308C03413BD
:102CE00006C0611104C08091BC01D801C3C04D87EA
:102CF0005E878D859E856A8B0E94F4146A8988237D
:102D0000E1F16623D1F12091BC01822F82958F7071
:102D100090E0029774F08091B7019091B801988784
:102D20008F831986DB86CA862C87CE0107960E9480
:102D3000B51486E0F801A7EBB1E001900D928A95F9
:102D4000E1F70E946C150E945E15FF24F394D6C033
:102D50004D875E878D859E850E94281A292F229592
:102D60002F7030E0223031050CF0BCC09F7009F0AC
:102D7000B6C0805E883008F4C1C0C8010E94B51496
:102D8000E4CFC816D90608F453C0F601E81BF90BC6
:102D9000CF01883C910508F450C0F12C7C2DD98AD4
:102DA000C88A89890E941E15E7EBF1E086E0DF0101
:102DB0001D928A95E9F70E945E15A0C0751314C094
:102DC000341312C0611110C08091BC01F8018583D9
:102DD000C8010E94B51486E0E7EBF1E0DF011D9227
:102DE0008A95E9F7FE2C8AC04D875E878D859E8582
:102DF0006A8B0E94F4146A89882309F4BECF662383
:102E000009F4BBCF2091BC01822F82958F7090E096
:102E100002970CF48ECF8091B7019091B8019A83FC
:102E200089831B82DD82CC822E83CE0101967FCFE7
:102E3000809590958C0D9D1DACCFF62E662309F4E0
:102E40009CCF75132EC034132CC02091BC0120FDE3
:102E50001FC0822F82958F70D9F0D80115962C93C0
:102E600015978F3049F08F5F982F9295907F822F22
:102E70008F70892B15968C93C8010E94B51486E03B
:102E8000F801A7EBB1E001900D928A95E1F793CF9D
:102E900086E0F801A7EBB1E001900D928A95E1F789
:102EA0002DC04D875E878D859E850E94F41481110B
:102EB00040CF8091BC0181608093BC01C8010E9419
:102EC000B5141CC0662309F458CF4D875E878D85E5
:102ED0009E850E94F414882309F44FCF2ACF8111D4
:102EE00048CF0CC0243031050CF047CF9F7009F457
:102EF00040CFF8019581907F09F03BCF8F2D6296EE
:102F00000FB6F894DEBF0FBECDBFDF91CF911F91FA
:102F10000F91FF90EF90DF90CF9008951F93CF9384
:102F2000DF93CDB7DEB72C970FB6F894DEBF0FBE98
:102F3000CDBF4F83588769877A878B879C87CE015F
:102F400007960E94C715882369F08F8198852A8586
:102F50003B85232BF1F19F3F09F063C08F3F09F0C0
:102F600060C037C086E0FE013796DE011196019001
:102F70000D928A95E1F76F817885EA85FB85309718
:102F800041F17F3F11F46F3F21F12091860130E044
:102F9000C9010196877099274091850150E08417F7
:102FA000950709F447C069837A83FD83EC8396E033
:102FB000929FD001939FB00D1124A957BE4FFE01DF
:102FC000319601900D929A95E1F7809386010E94C7
:102FD0003D1516E080918501909186018917C1F118
:102FE000189FC001112489579E4F0E94C71588233E
:102FF00079F1E09185011E9FF0011124E957FE4F00
:103000004081518162817381848195810E942D1557
:103010008091850190E001968770992780938501C2
:10302000D9CF4F81588569857A858B859C850E948B
:103030002D15CFCF0E94F0141092860110928501B9
:10304000E7EBF1E086E0DF011D928A95E9F7C1CF59
:103050002C960FB6F894DEBF0FBECDBFDF91CF9197
:103060001F910895EF92FF920F931F93CF93DF93D9
:103070008C01892B09F46CC0F12CEE24E394E80157
:103080002196F8018491843740F4843008F051C0CF
:10309000813081F0823019F15BC0853709F444C07A
:1030A000A8F19CE7980F903708F052C08F770E94E4
:1030B0003B1241C00E5F1F4FFE01C49180E28C0F96
:1030C000883048F4C7708E2D01C0880FCA95EAF782
:1030D0000E940E1B14C08C2F0E9473112DC00E5F16
:1030E0001F4FFE01C49180E28C0F883058F4C770E6
:1030F0008E2D01C0880FCA95EAF70E94141B0E940A
:10310000351B1AC08C2F0E943B1216C00E5F1F4F3A
:10311000FE01C491CC2381F08FE99FE00197F1F784
:1031200000C00000C150F6CF0E5F1F4FFE01F490AB
:1031300003C00E9473118E018F2D882309F49FCF45
:10314000EFE9FFE03197F1F700C000008150F5CFC3
:10315000DF91CF911F910F91FF90EF900895089507
:103160006093C1017093C2018093C3019093C40125
:103170000C94DC140F931F930091C1011091C201B4
:103180002091C3013091C401DC01CB01802B912B34
:10319000A22BB32B8093C1019093C201A093C301D2
:1031A000B093C4011F910F910C94DC140F931F93E3
:1031B0000091C1011091C2012091C3013091C4015D
:1031C000DC01CB0180239123A223B3238093C1018F
:1031D0009093C201A093C301B093C4011F910F91BA
:1031E0000C94DC140F931F930091C1011091C20144
:1031F0002091C3013091C401DC01CB0180279127CC
:10320000A227B3278093C1019093C201A093C30169
:10321000B093C4011F910F910C94DC141092BD0166
:103220001092BE011092BF011092C0010C94DC14E8
:1032300041E050E060E070E004C0440F551F661F9D
:10324000771F8A95D2F74093BD015093BE016093DA
:10325000BF017093C0010C94DC1441E050E060E0C9
:1032600070E004C0440F551F661F771F8A95D2F780
:103270008091BD019091BE01A091BF01B091C001AC
:10328000482B592B6A2B7B2B4093BD015093BE01D9
:103290006093BF017093C0010C94DC1441E050E0D6
:1032A00060E070E004C0440F551F661F771F8A95C9
:1032B000D2F740955095609570958091BD019091A1
:1032C000BE01A091BF01B091C001482359236A23D8
:1032D0007B234093BD015093BE016093BF01709367
:1032E000C0010C94DC1441E050E060E070E004C0E8
:1032F000440F551F661F771F8A95D2F78091BD0135
:103300009091BE01A091BF01B091C00148275927FB
:103310006A277B274093BD015093BE016093BF0194
:103320007093C0010C94DC140F931F930091BD01A6
:103330001091BE012091BF013091C001DC01CB0191
:10334000802B912BA22BB32B8093BD019093BE01B8
:10335000A093BF01B093C0011F910F910C94DC1496
:103360000F931F930091BD011091BE012091BF01E9
:103370003091C001DC01CB0180239123A223B32330
:103380008093BD019093BE01A093BF01B093C00193
:103390001F910F910C94DC140F931F930091BD01AA
:1033A0001091BE012091BF013091C001DC01CB0121
:1033B00080279127A227B3278093BD019093BE0158
:1033C000A093BF01B093C0011F910F910C94DC1426
:1033D0000895CF92DF92EF92FF920F931F93CF93B6
:1033E000DF938C01C090C101D090C201E090C30175
:1033F000F090C4018091BD019091BE01A091BF01E8
:10340000B091C001C82AD92AEA2AFB2ACFE1D0E02C
:10341000D701C6010C2E04C0B695A7959795879540
:103420000A94D2F780FF06C0B8018C2F0E94B5081D
:10343000019721F4219760F780E001C08C2FDF9184
:10344000CF911F910F91FF90EF90DF90CF90089553
:10345000CF93DF93EC010E94E919BE010E94B508E9
:10346000DF91CF910895CB010E94281A0895809191
:10347000C50185958595859508958091C5018770CD
:10348000089598E0899F90011124262B2093C5016F
:103490000C942D192091C501809582238093C5013C
:1034A000982F977069F430E0482F552747FD5095C5
:1034B0002417350729F08595859585950C944E1927
:1034C00008959091C501977081E009F480E0089516
:1034D00090910C01992321F090910D01911109C057
:1034E00020910E0130910F01F90132969FEF40E0DB
:1034F0001FC0982F9695969596959F3050F5E09120
:103500000E01F0910F01E90FF11D877021E030E00D
:10351000A90102C0440F551F8A95E2F7CA019181A3
:10352000892B818308959F3F39F04F5F4E3041F0E2
:1035300051915813F8CF0DC05111F7CF942FF5CFFB
:103540009F3F39F0F901E90FF11D97FDFA9582834C
:103550000895089590910C01992321F090910D0107
:10356000911109C020910E0130910F01F90132969D
:10357000205F3F4F1FC0982F9695969596959F3048
:10358000F0F4E0910E01F0910F01E90FF11D877049
:1035900021E030E0A90102C0440F551F8A95E2F7EF
:1035A000CA01809591818923818308953196E2171C
:1035B000F30729F090819813F9CF1082F7CF08957F
:1035C00081E090E0E0910E01F0910F01E80FF91F0A
:1035D0001082019680319105A9F708959091D90143
:1035E000892B8093D901089580959091D9018923E1
:1035F0008093D90108951092D90108959091D8012E
:10360000892B8093D801089580959091D8018923C2
:103610008093D80108951092D80108959091D70110
:10362000892B8093D701089580959091D7018923A4
:103630008093D70108951092D70108958093C60111
:1036400008951092C601089580910E0190910F0186
:10365000FC0131969C01205F3F4F80E091919111D8
:103660008F5FE217F307D1F70895E0910E01F09113
:103670000F018091D9018083E0910E01F0910F013B
:1036800090818091D801892B8083E0910E01F09187
:103690000F0190818091D701892B80838091C60191
:1036A000882361F0E0910E01F0910F019081892B48
:1036B00080830E94241B81111092C60180910E010B
:1036C00090910F010C94631020E0009739F0AC0149
:1036D00041505109842395232F5FF7CF822F0895FE
:1036E000CF92DF92EF92FF926C01EE24FF24C1147F
:1036F000D104E104F10421F0C701B60120E101C0C9
:1037000020E0C72ED82EE92EFF24C114D104E104F5
:10371000F10419F0285FC701B6016B017C0154E088
:10372000F694E794D794C7945A95D1F7C114D1046D
:10373000E104F10419F02C5FC701B6016B017C01B3
:1037400042E0F694E794D794C7944A95D1F7C11410
:10375000D104E104F10419F02E5FC701B601DC01C8
:10376000CB01B695A79597958795892B8A2B8B2B9F
:1037700009F02F5F822FFF90EF90DF90CF90089598
:103780008091F101843021F11092DB0120E488E185
:1037900090E00FB6F894A895809360000FBE209338
:1037A000600080E00E94500983B7817F846083BFFE
:1037B00083B7816083BF7894889583B78E7F83BFFA
:1037C00088E10FB6F89480936000109260000FBEFD
:1037D0000895089508950E94E91B0E94B0040E9474
:1037E000EA1B0E94A50591E0811101C090E0892F9C
:1037F00008950E94F0140E9457100C94500982E022
:1038000084BD93E095BD9AEF97BD80936E000895B7
:103810002FB7F8948091DC019091DD01A091DE0139
:10382000B091DF012FBF0895CF92DF92EF92FF9208
:103830000F931F932FB7F8944091DC015091DD0155
:103840006091DE017091DF012FBF6A017B01EE24E0
:10385000FF248C0120E030E0C016D106E206F3061A
:1038600010F4415051099A01281B390BC9011F91CD
:103870000F91FF90EF90DF90CF9008951F920F92DD
:103880000FB60F9211248F939F93AF93BF938091A4
:10389000DC019091DD01A091DE01B091DF01019684
:1038A000A11DB11D8093DC019093DD01A093DE0189
:1038B000B093DF01BF91AF919F918F910F900FBE99
:1038C0000F901F9018950E94540DF8942FEF87EADF
:1038D00091E6215080409040E1F700C0000087E071
:1038E00090EBDC018093FB019093FC01A093FD0120
:1038F000B093FE019CE088E10FB6F894A895809300
:1039000060000FBE90936000FFCFEF92FF920F9385
:103910001F93CF93DF93D82FCDE08C2F0E949E056D
:1039200005E010E0E82EF12CC701002E02C09595AD
:1039300087950A94E2F780FF09C0602F7C2F80E012
:103940000E946106D81302C081E006C0015011092F
:1039500058F7C15010F780E0DF91CF911F910F9180
:10396000FF90EF900895CF93C82F8CE20E94851CA2
:10397000882321F08C2FCF910C94851C80E0CF916F
:103980000895CF930E94081E811102C00E94EE1D6F
:10399000C5E6C15049F00E94B0048FE39CE901974D
:1039A000F1F700C00000F5CF89E20E94B31C81113D
:1039B00013C18AE20E94B31C81110E94EE1D85E0B2
:1039C0000E94B31C81110E94631C0E94131E8093ED
:1039D000DA0187E00E94B31C8823A9F18BE10E94E1
:1039E000B31C882351F08091DA0181FB222720F952
:1039F00091E0922790FB81F90EC08EE00E94B31CEB
:103A0000882361F08091DA0182FB222720F991E07E
:103A1000922790FB82F98093DA0115C080E10E9421
:103A2000B31C9091DA01882341F093FB222720F9FF
:103A300081E0822780FB93F904C0892F809580FB69
:103A400090F99093DA018091DA010E94171E0E948A
:103A5000251E8093FA0180EE0E94B31C882341F05A
:103A60008091FA01982F909590FB80F98093FA014C
:103A700089E30E94B31C882359F08091FA0181FBED
:103A8000222720F991E0922790FB81F98093FA0197
:103A900082EE0E94B31C882359F08091FA0182FBC8
:103AA000222720F991E0922790FB82F98093FA0176
:103AB00086EE0E94B31C882359F08091FA0183FBA3
:103AC000222720F991E0922790FB83F98093FA0155
:103AD00083EE0E94B31C882359F08091FA0184FB85
:103AE000222720F991E0922790FB84F98093FA0134
:103AF00085E30E94B31C882359F08091FA0185FB6D
:103B0000222720F991E0922790FB85F98093FA0112
:103B100081E30E94B31C882359F08091FA0186FB4F
:103B2000222720F991E0922790FB86F98093FA01F1
:103B300081E10E94B31C882359F08091FA0187FB30
:103B4000222720F991E0922790FB87F98093FA01D0
:103B50008091FA010E94291E8091FA0187FB882733
:103B600080F980930D0187E20E94B31CC82F8EE17B
:103B70000E94B31C8111C2608FE10E94B31C8111AD
:103B8000C46080E20E94B31C8111C86081E20E947F
:103B9000B31C8111C06182E20E94B31C8111C0621A
:103BA00083E20E94B31C8111C06484E20E94B31CB2
:103BB000882311F0C06802C0CC2329F08C2F0E940A
:103BC000201E6C2F03C00E941C1E682F70E080E036
:103BD00090E0CF910C94B018CF9108956DEE7EEFE8
:103BE00080E090E00E945A2460E082E090E00E9431
:103BF000482460E083E090E00E94482460E084E094
:103C000090E00E94482460E085E090E00C94482415
:103C100080E090E00E94422421E08D3E9E4F09F01A
:103C200020E0822F089582E090E00C943A24682FDF
:103C300082E090E00C94482483E090E00C943A24D5
:103C4000682F83E090E00C94482484E090E00C948A
:103C50003A24682F84E090E00C9448248091E2019B
:103C600080FF0BC06091130185E0689FB0011124B3
:103C700075956795759567952BC081FF09C0609113
:103C8000130185E0689FB00111247595679520C0E8
:103C900082FF07C06091130185E0689FB001112485
:103CA00017C09091E3019923D1F06091120196170A
:103CB00088F72091130185E0289F90011124929F9D
:103CC000A001939F500D112470E0CA010E940C24A2
:103CD0006038710540F46115710539F002C065E086
:103CE00070E0862F08958FE7089581E00895809110
:103CF000E20180FF08C06091110170E07595679541
:103D00007595679521C081FF06C06091110170E033
:103D10007595679519C082FF04C06091110170E02C
:103D200010C09091E3019923C1F0609110019617A2
:103D3000A0F780911101899FC001112470E00E94B9
:103D40000C246038710528F46115710521F0862F67
:103D500008958FE7089581E0089561E070E0F4CF61
:103D6000803F21F40E942E1E819504C0813F29F4DA
:103D70000E942E1E8093E6010895823F21F40E9446
:103D80002E1E819504C0833F29F40E942E1E80932D
:103D9000E5010895893F19F40E94771E05C08A3F06
:103DA00031F40E94771E81958093E70108958B3F3F
:103DB00021F40E94771E819504C08C3F29F40E9453
:103DC000771E8093E8010895843F21F48091E401F7
:103DD000816017C0853F21F48091E401826011C0A9
:103DE000863F21F48091E40184600BC0873F21F479
:103DF0008091E401886005C0883F31F48091E4013E
:103E000080618093E40108958D3F21F48091E20167
:103E100081600BC08E3F21F48091E201826005C079
:103E20008F3F29F48091E20184608093E20108953C
:103E3000803F39F48091E60187FF6CC01092E60163
:103E400069C0813F29F48091E6011816BCF362C075
:103E50009091E501823F29F497FF5CC01092E50143
:103E600059C0833F19F41916CCF354C0893F41F46B
:103E70008091E70118160CF04DC01092E7014AC07E
:103E80008A3F29F48091E70187FF44C0F6CF8B3F3A
:103E900039F48091E80187FF3DC01092E8013AC0F3
:103EA0008C3F29F48091E8011816BCF333C0843F9D
:103EB00021F48091E4018E7F17C0853F21F4809129
:103EC000E4018D7F11C0863F21F48091E4018B7F56
:103ED0000BC0873F21F48091E401877F05C0883FB4
:103EE00031F48091E4018F7E8093E40113C08D3F13
:103EF00021F48091E2018E7F0BC08E3F21F48091EE
:103F0000E2018D7F05C08F3F29F48091E2018B7F14
:103F10008093E2018091E50181110EC08091E6015C
:103F200081110AC08091E701811106C08091E801EA
:103F3000811102C01092E301089584EE91E00E9485
:103F40006E100E94081C9093E1018093E001089597
:103F50001F93CF93DF938091E0019091E1010E9444
:103F6000141CAC019091E301992321F020911401DC
:103F700030E006C0209115018AE0289F90011124AD
:103F80004217530708F486C08091E501C091E6010D
:103F9000D091E7011091E801811107C0C11176C0ED
:103FA000D11174C0111172C075C09F3F19F09F5F8D
:103FB0009093E301181624F40E942E1E8093E501CD
:103FC0008091E50187FF05C00E942E1E8195809398
:103FD000E5011C1624F40E942E1E8093E6018091B8
:103FE000E60187FF05C00E942E1E81958093E601A1
:103FF0006091E501662339F1C091E601CC2319F106
:10400000772767FD7095872F972F0E941D2323E345
:1040100033E343E35FE30E9481230E94EA2260933B
:10402000E5016C2F772767FD7095872F972F0E94EA
:104030001D2323E333E343E35FE30E9481230E94D4
:10404000EA226093E6011D1624F40E94771E8093F5
:10405000E7018091E70187FF05C00E94771E8195E7
:104060008093E701111624F40E94771E8093E801E3
:104070008091E80187FF05C00E94771E819580939B
:10408000E801DF91CF911F910C949D1F9F3F09F094
:104090008ECF96CFDF91CF911F910895E4EEF1E09E
:1040A00085E0DF011D928A95E9F71092E3011092F5
:1040B000E2010895833081F128F4813059F0823093
:1040C000D1F00895853009F449C0B8F1863009F47B
:1040D00056C0089580911501262F30E0280F311D1C
:1040E0002F3F310524F4680F6093150108958FEF79
:1040F00080931501089580911401262F30E0280F38
:10410000311D2F3F310524F4680F60931401089589
:104110008FEF80931401089580911301262F30E0D2
:10412000280F311D2F3F310524F4680F60931301D0
:1041300008958FEF80931301089580911201262F27
:1041400030E0280F311D2F3F310524F4680F6093B4
:10415000120108958FEF809312010895809111014B
:10416000262F30E0280F311D2F3F310524F4680F32
:104170006093110108958FEF80931101089580914C
:104180001001262F30E0280F311D2F3F310524F478
:10419000680F6093100108958FEF809310010895C8
:1041A000833011F128F4813049F0823091F0089584
:1041B000853081F120F18630C1F10895809115019B
:1041C000681720F4861B809315010895109215013D
:1041D000089580911401681720F4861B80931401C0
:1041E000089510921401089580911301681720F426
:1041F000861B8093130108951092130108958091F6
:104200001201681720F4861B809312010895109202
:104210001201089580911101681720F4861B809384
:1042200011010895109211010895809110016817ED
:1042300020F4861B809310010895109210010895B8
:104240000F931F938D3109F46BC008F03FC08E307F
:1042500009F47FC0C0F4873009F469C068F486307F
:1042600009F0B1C08091DA01817F8E7F8093DA01FD
:1042700081E08093EA01A8C0883009F4A2C08B30A5
:1042800009F49FC0A0C0863109F49BC078F4803146
:1042900009F472C0813109F096C00E94F014909127
:1042A0000D0181E0892780930D018BC0893109F4CC
:1042B00088C08B3109F087C08091DA0181FB222709
:1042C00020F991E0922790FB81F94CC0853309F4E5
:1042D00070C048F4873209F46CC008F459C08932C0
:1042E00009F467C070C0833438F48A3308F04EC0D4
:1042F000883309F466C067C0833409F45AC088342F
:1043000009F061C00E94F0140FEF13ED20E301509B
:1043100010402040E1F700C000000E94631C51C023
:104320000E94A4220E9457100E9450094AC09091F6
:10433000DA01892F8095817080FB90F929F09660D1
:1043400098609093DA0140C0997F977F9093DA014B
:1043500038C08091DA0182FB222720F991E0922770
:1043600090FB82F98093DA01992359F18091DA0167
:1043700081608093DA0125C08091DA0183FB2227D6
:1043800020F991E0922790FB83F9ECCF895301C08B
:104390008D5141E050E060E070E08A019B0104C073
:1043A000000F111F221F331F8A95D2F7C901B801D0
:1043B00004C061E070E080E090E00E94B0180E94CC
:1043C000F01481E001C080E01F910F91089580E01A
:1043D000089580E00895CF93C82F8091EA0181303D
:1043E00079F018F08230E9F187C0E0910E01F09188
:1043F0000F018081813169F0823209F07FC009C0EC
:10440000E0910E01F0910F018081813111F0823233
:1044100061F48C2F0E94E721811104C08C2F0E942F
:1044200020211DC081E090E01AC08C2F0E94E9215C
:10443000811114C0C43179F048F4CB3079F0C03127
:1044400009F060C082E08093EA0108C0C93219F027
:10445000C83321F057C01092EA0154C081E0817046
:1044600053C0C93289F118F5C43171F1A8F4C730CD
:1044700009F046C08AE08093150194E190931401FD
:1044800093E0909313018093120188E080931101CF
:1044900088E28093100134C0CE51C63088F5EC2FED
:1044A000F0E0E65DFE4F80818093E90129C0CE34C3
:1044B000E9F020F4CB3421F56AE013C0C13579F07E
:1044C000C235F1F461E00DC08091E901882319F053
:1044D0001092E90115C081E08093EA0115C061E006
:1044E00006C08091E9010E945A200AC06AE08091CA
:1044F000E9010E94D02004C01092EA0180E004C0CB
:1045000081E002C080E0ABCFCF910895E1E8F0E018
:104510008081886080838081816080838FB7F894F8
:1045200093E09093890090ED909388008FBF089559
:10453000EFE6F0E08081826080830895EFE6F0E0AE
:1045400080818D7F80830895EFE6F0E0908182E0A6
:104550008927808308951F920F920FB60F9211241E
:104560002F933F934F935F936F937F938F939F937B
:10457000AF93BF93EF93FF938091EB019091EC0188
:1045800001969093EC018093EB01811103C082E0CE
:104590000E945009E091EC01E695E695F0E0EB59B8
:1045A000FA4FE4918091EB018E1303C080E00E94EA
:1045B0005009FF91EF91BF91AF919F918F917F91A2
:1045C0006F915F914F913F912F910F900FBE0F9080
:1045D0001F90189504D06894B1118DC0089570D0C3
:1045E00088F09F5790F0B92F9927B751A0F0D1F0DC
:1045F000660F771F881F991F1AF0BA95C9F712C066
:10460000B13081F077D0B1E0089574C0672F782F72
:104610008827B85F39F0B93FCCF3869577956795D1
:10462000B395D9F73EF490958095709561957F4F3D
:104630008F4F9F4F0895E89409C097FB3EF49095E3
:104640008095709561957F4F8F4F9F4F9923A9F06B
:10465000F92F96E9BB279395F695879577956795FA
:10466000B795F111F8CFFAF4BB0F11F460FF1BC03E
:104670006F5F7F4F8F4F9F4F16C0882311F096E9D1
:1046800011C0772321F09EE8872F762F05C066237F
:1046900071F096E8862F70E060E02AF09A95660F38
:1046A000771F881FDAF7880F9695879597F90895F1
:1046B00057FD9058440F551F59F05F3F71F04795D3
:1046C000880F97FB991F61F09F3F79F087950895B8
:1046D000121613061406551FF2CF4695F1DF08C0D7
:1046E000161617061806991FF1CF869571056105F4
:1046F00008940895E894BB2766277727CB0197F99C
:1047000008950BD078C069D028F06ED018F09523AA
:1047100009F05AC05FC01124EECFCADFA0F3959F05
:10472000D1F3950F50E0551F629FF001729FBB2798
:10473000F00DB11D639FAA27F00DB11DAA1F649F44
:104740006627B00DA11D661F829F2227B00DA11DF7
:10475000621F739FB00DA11D621F839FA00D611D7D
:10476000221F749F3327A00D611D231F849F600D9E
:10477000211D822F762F6A2F11249F5750408AF0D7
:10478000E1F088234AF0EE0FFF1FBB1F661F771F63
:10479000881F91505040A9F79E3F510570F014C0FA
:1047A000AACF5F3FECF3983EDCF38695779567954B
:1047B000B795F795E7959F5FC1F7FE2B880F911D81
:1047C0009695879597F9089597F99F6780E870E027
:1047D00060E008959FEF80EC089500240A94161677
:1047E000170618060906089500240A9412161306DF
:1047F000140605060895092E0394000C11F488236D
:1048000052F0BB0F40F4BF2B11F460FF04C06F5F88
:104810007F4F8F4F9F4F089597FB072E16F40094FC
:1048200007D077FD09D00E94262407FC05D03EF46E
:10483000909581959F4F0895709561957F4F08954C
:10484000EE0FFF1F0590F491E02D0994AA1BBB1BEE
:1048500051E107C0AA1FBB1FA617B70710F0A61B80
:10486000B70B881F991F5A95A9F780959095BC01A1
:10487000CD010895F999FECF92BD81BDF89A99278F
:1048800080B50895A8E1B0E042E050E00C946224C5
:10489000262FF999FECF92BD81BDF89A019700B4F9
:1048A000021639F01FBA20BD0FB6F894FA9AF99A99
:1048B0000FBE08950196272F0E9449240C94482486
:1048C000DC01CB01FC01F999FECF06C0F2BDE1BDD0
:1048D000F89A319600B40D9241505040B8F70895BF
:0448E000F894FFCF7A
:1048E40020025209E009BD09890955090101C701DE
:1048F40028080A03140A3F4D36392605D904A304AF
:104904006A04FD0316042F04480401020304050687
:044914000708090087
:00000001FF
